:100000000C94AC000C94D4000C94D4000C94D40048
:100010000C94D4000C94D4000C94D4000C94D40010
:100020000C94D4000C94D4000C9426040C949804E2
:100030000C94D4000C94D4000C94D4000C94D400F0
:100040000C94D4000C94D4000C94D4000C94D400E0
:100050000C94D4000C94D4000C94D4000C94C806D6
:100060000C94D4000C94D4000C94D4000C94D400C0
:100070000C94D4000C94D4000C94D4000C94D400B0
:100080000C94D4000C94D4000C94D4000C94D400A0
:100090000C94D4000C94D4000C94D4000C94D40090
:1000A0000C94D4000C94D4000C94D40005010904E1
:1000B000A101A100050919012909150025019509CA
:1000C0007501810295017507810305010901A100F0
:1000D0000930093115FF2501950275088102C0C05C
:1000E000C0080B0002020201000904000001020224
:1000F000000005240010010524010101042402066A
:1001000005240600010705810310004009040100D1
:10011000020A0000000705020240000007058302F2
:100120004000000403090412010002EF02014041F3
:1001300023368000010102030141726475696E6F0C
:10014000204C4C430041726475696E6F204C656FA2
:100150006E6172646F004F0711241FBECFEFDAE0AB
:10016000DEBFCDBF11E0A0E0B1E0EAE0F3E102C004
:1001700005900D92A034B107D9F721E0A0E4B1E0D9
:1001800001C01D92AC3DB207E1F710E0CCEAD0E02F
:1001900004C02197FE010E947109CB3AD107C9F72B
:1001A0000E94F0070C9483090C940000FC018091DC
:1001B0006701811103C08FEF9FEF08959FB7F894F7
:1001C00082E08093E9002091F20030E012161306DD
:1001D00014F421E030E02115310559F0289884E627
:1001E000809366018091F10080838091F2008823E2
:1001F00019F09FBFC90108958BE68093E800F9CFFD
:10020000CF92DF92EF92FF920F931F93CF93DF93E2
:100210006C017A018B01C0E0D0E0CE15DF0589F0DA
:10022000D8016D918D01D601ED91FC910190F08185
:10023000E02DC6010995892B11F47E0102C021969B
:10024000ECCFC701DF91CF911F910F91FF90EF90FD
:10025000DF90CF900895CF93DF931F92CDB7DEB795
:100260006983DC01ED91FC910280F381E02D41E096
:1002700050E0BE016F5F7F4F09950F90DF91CF91E6
:10028000089583E08093E9008091F200882319F0BB
:100290008AE38093E8000895CF93DF931F92CDB750
:1002A000DEB7FC018485958597FD05C02FEF3FEFF4
:1002B000358724870BC0CE0101960E94D600019796
:1002C00019F4898190E002C08FEF9FEF0F90DF91CA
:1002D000CF9108950F931F93CF93DF931F92CDB7C4
:1002E000DEB78C01FC018485958597FF0EC0CE0199
:1002F00001960E94D600019719F4298130E002C0CE
:100300002FEF3FEFF80135872487F8018485958525
:100310000F90DF91CF911F910F910895FC0184857B
:10032000958597FD0BC09FB7F89482E08093E90014
:100330008091F2009FBF90E0019608959FB7F894D6
:1003400082E08093E9008091F2009FBF90E00895E1
:10035000089580E090E00895409157015091580130
:10036000209155013091560142175307B4F49091F2
:10037000E8009570E1F39091E80092FD19C0809338
:10038000F100809157019091580101968F73992740
:10039000892B19F48EEF8093E8008091570190919A
:1003A00058010196909358018093570181E0089578
:1003B00080E00895DF92EF92FF920F931F93CF9307
:1003C000DF93D82E8A017B01E40EF51EEB01CE15DA
:1003D000DF0571F0D7FE03C0FE01849101C0888162
:1003E0000E94AC0121968111F2CF8FEF9FEF01C0E7
:1003F000C801DF91CF911F910F91FF90EF90DF9097
:1004000008952FB7F89487708093E9009091E800E1
:10041000892F807295FF04C09091F20080E4891BBF
:100420002FBF089583E00E94010290E0089561507B
:1004300030F02091F100FC0120830196F8CF28983C
:1004400084E680936601089580914D0181110DC06D
:1004500082E08093490184E080934A0110924C012C
:1004600010924B0181E080934D0189E491E0089561
:100470000F931F93CF93DF931F92CDB7DEB782E028
:10048000898342E450E061EE70E080E80E94DA0186
:100490000E942402DC0112960D911C911397011504
:1004A000110569F0D801ED91FC910280F381E02DF6
:1004B000BE016F5F7F4FC801099597FF07C0898113
:1004C0000F90DF91CF911F910F910895F801008552
:1004D0001185E5CF3FB7F894809145019091460191
:1004E000A0914701B091480126B5A89B05C02F3FB8
:1004F00019F00196A11DB11D3FBFBA2FA92F982F4A
:100500008827820F911DA11DB11DBC01CD0142E0C4
:10051000660F771F881F991F4A95D1F708958F920C
:100520009F92AF92BF92CF92DF92EF92FF926B01B8
:100530007C010E946A024B015C01C114D104E104F8
:10054000F104F1F00E946A02DC01CB0188199909DB
:10055000AA09BB09883E9340A105B10570F321E0CB
:10056000C21AD108E108F10888EE880E83E0981ECF
:10057000A11CB11CC114D104E104F10419F7DDCFB1
:10058000FF90EF90DF90CF90BF90AF909F908F90B3
:1005900008957F928F929F92AF92BF92CF92DF92F7
:1005A000EF92FF920F931F93CF93DF93C82E8B018F
:1005B0007A0180916701811103C08FEF9FEF75C0B1
:1005C00080915B0180FF05C08091E0008260809394
:1005D000E000CE2DDF2DD12C8AEF882E8C2D877058
:1005E000B82E8C2D8072A82E8C2D8074982E9AE3B4
:1005F000792E209709F452C08C2D0E940102282FD9
:1006000081110AC08A948820C1F261E070E080E024
:1006100090E00E948F02EDCF90E0C817D9070CF44C
:100620002C2F3FB7F894B092E9008091E80085FF45
:1006300033C0822F90E0C81BD90BAA2029F021508B
:10064000A8F01092F100FBCFF801C7FE07C02150BF
:1006500058F044914093F1003196F9CF215020F0A9
:1006600041914093F100FACF080F191FDD2019F0D6
:100670007092E8000AC08091E80085FD08C0709281
:10068000E800DD24D394209739F0D12C05C02097C1
:1006900019F491107092E8003FBFABCFD110ACCFEE
:1006A0005D9884E680935901C701DF91CF911F9136
:1006B0000F91FF90EF90DF90CF90BF90AF909F9001
:1006C0008F907F900895CF93DF93EC0180910B0181
:1006D000882331F083E00E94C9021816190634F00D
:1006E00081E090E09B838A8380E090E0DF91CF916E
:1006F0000895DC01FB0112968C91129790E0248101
:10070000358182179307D1F491818081813A31F448
:1007100081E0913091F0933089F411C0813271F40D
:100720009B3021F482811C968C9305C09A3031F461
:1007300082811D968C9381E00895089580E008954C
:10074000FB0120812138B9F423812232A1F4DC019C
:1007500012962C91129730E044815581421753072D
:1007600051F421E01C962C9345E350E06CEA70E0D4
:1007700080E80C94DA0180E090E00895CF93DF9355
:10078000CDB7DEB769970FB6F894DEBF0FBECDBF09
:10079000FC01DB019C919F5F9C93BE016F5F7F4FCB
:1007A00089E1DB011D928A95E9F729E0298384E03C
:1007B0008A8391E09D8383E08E832A8721E22B87C1
:1007C0009C879D879F8722E2288B25E3298B27E042
:1007D0002B8B25E02C8B8E8B20E430E0388F2F8BF9
:1007E000998F82818B83838180688D8B49E150E072
:1007F00080E00E94DA0169960FB6F894DEBF0FBE62
:10080000CDBFDF91CF910895FC0182818F5BFB0109
:10081000808381E008950E947709CF93DF93EB01F5
:10082000FC0180859185892B69F461E371E0CE013B
:100830000E947C09FE0101900020E9F731978E2F7C
:100840008C1B01C080E0DF91CF9108951F920F9221
:100850000FB60F9211248F939F938091E100909196
:10086000E100937F9093E10083FF0FC01092E900B5
:1008700091E09093EB001092EC0092E39093ED00E6
:100880001092670198E09093F00082FF20C093E0FF
:100890009093E9009091F200992319F09AE39093D4
:1008A000E80090915901992339F0909159019150A4
:1008B00090935901992389F190916601992339F018
:1008C00090916601915090936601992341F184FFC4
:1008D00010C08091E2008E7E81608093E200809162
:1008E000E1008F7E8093E10080915B018E7E8061CC
:1008F00011C080FF16C08091E2008E7E80618093DF
:10090000E2008091E1008E7E8093E10080915B01A6
:100910008E7E816080935B0104C05D9ACDCF289A62
:10092000D6CF9F918F910F900FBE0F901F9018956B
:100930001F920F920FB60F921124CF92DF92EF9277
:10094000FF920F931F932F933F934F935F936F9358
:100950007F938F939F93AF93BF93EF93FF93CF9327
:10096000DF93CDB7DEB76C97DEBFCDBF1092E90045
:100970008091E80083FFEDC168E0CE0145960E94BA
:10098000170282EF8093E8008D8987FF05C0909160
:10099000E80090FFFCCF03C09EEF9093E800982FF3
:1009A000907609F0C6C09E892F89188D91110CC0D0
:1009B000803829F480915C018093F10002C010928C
:1009C000F1001092F10048C1422F50E0512B9130BC
:1009D00051F4811141C14130510509F03DC180916F
:1009E0005C018D7F0BC0933061F4811135C14130C2
:1009F000510509F031C180915C01826080935C01F6
:100A00002BC1953041F48091E80080FFFCCF206835
:100A10002093E30021C1963009F05FC0EB8CFC8C81
:100A20001092E9001092580110925701123091F57E
:100A300010925601109255010E94380299E0BE01B1
:100A40006F5F7F4FDB01E92F1D92EA95E9F79983EC
:100A50001A8391E09E8390EA98879AEF9987209174
:100A6000570130915801275F3F4F3C832B838D8383
:100A70001092E9001092580110925701F09256011D
:100A8000E092550149E050E080E00E94DA010E94C6
:100A90003802E2C0F0925601E09255010E94240211
:100AA000DC011296ED90FC901397E114F10409F427
:100AB000C0C0D701ED91FC910480F581E02DBE010D
:100AC0006B5E7F4FC7010995009719F00CF0C4C009
:100AD000C7C0F701E084F184E8CF973009F4C0C0C3
:100AE000983021F481E08093F100B6C0993009F08C
:100AF000B3C0837009F0B4C0EDE0F1E081E021E023
:100B000036E39081992361F08093E9002093EB0014
:100B100091919093EC003093ED008F5F873089F7CF
:100B20008EE78093EA001092EA008F898093670134
:100B300093C08B8D9C8D1092E900109258011092F9
:100B400057019093560180935501898D811156C0AC
:100B50008E899D89913A59F4813209F081C047E02C
:100B600050E064E071E080E00E94DA0175C09132EB
:100B700009F076C0833289F4888D90E0982F882719
:100B80002F89822BA0E0B0E08093000190930101B7
:100B9000A0930201B09303015FC0803269F4809199
:100BA000E80082FFFCCF67E084E091E00E9417023A
:100BB0008BEF8093E80006C0823209F04DC08F8928
:100BC00080930B0180915A01882319F0EEEFFAE02F
:100BD00002C0E0E0F8E08091040190910501A0914D
:100BE0000601B0910701803B9440A105B10509F0D1
:100BF0007BC080910B0180FF93C076C00E942402CD
:100C0000DC0112960D911C9113970115110541F10C
:100C1000D801ED91FC910190F081E02DBE016B5E59
:100C20007F4FC8010995811117C0F8010085118512
:100C3000ECCF113009F44EC0133091F48F89882322
:100C400009F445C0823081F440E860E185E491E038
:100C50000E941207882321F08EEF8093E80079C06C
:100C600081E28093EB0075C0813029F440E86BE0AD
:100C700089E391E0EDCF833099F70E942402DC01F3
:100C80001296ED90FC9013978E010F5F1F4F680135
:100C9000E114F10479F0D701ED91FC910680F78120
:100CA000E02DB801C7010995080F111DF701E08477
:100CB000F184EECFD8011C92F60101900020E9F7F3
:100CC0003197BF016C197D0940E0C601C1CF63E2D5
:100CD00071E002C067E271E06115710509F2FB0184
:100CE000449150E080E840CF0FB6F894A8958091E9
:100CF0006000886180936000109260000FBEA8952C
:100D0000EE3F2AE0F20739F08091FE0A9091FF0A47
:100D100091838083A1CF1092FF0A1092FE0A9CCF8C
:100D2000EE3F8AE0F80731F0808191819093FF0ACD
:100D30008093FE0A87E797E7918380839BE088E1B1
:100D40000FB6F894A895809360000FBE9093600052
:100D500083CF6C960FB6F894DEBF0FBECDBFDF9188
:100D6000CF91FF91EF91BF91AF919F918F917F9123
:100D70006F915F914F913F912F911F910F91FF9034
:100D8000EF90DF90CF900F900FBE0F901F901895AF
:100D90001F920F920FB60F9211242F933F938F93B0
:100DA0009F93AF93BF938091410190914201A09195
:100DB0004301B09144013091400123E0230F2D37CE
:100DC00020F40196A11DB11D05C026E8230F02964F
:100DD000A11DB11D209340018093410190934201D8
:100DE000A0934301B0934401809145019091460145
:100DF000A0914701B09148010196A11DB11D8093BA
:100E0000450190934601A0934701B0934801BF91DB
:100E1000AF919F918F913F912F910F900FBE0F90A7
:100E20001F901895CF92DF92EF92FF920F931F932E
:100E3000CF93DF931F92CDB7DEB7182F062FE42E86
:100E4000862F880F8E5F99830E94AC0183E00E94F9
:100E5000AC01F12EC12E9981D92E8C2D8F198017BE
:100E600098F4F601E7FE02C0849101C080810E94DF
:100E7000AC01182F80E00E94AC018123FFEFCF1A54
:100E8000DF0A8111EACF01C081E00F90DF91CF919D
:100E90001F910F91FF90EF90DF90CF9008958F9268
:100EA0009F92AF92BF92CF92DF92EF92FF920F93F9
:100EB0001F93CF93DF9310926B0110926A0188EE1B
:100EC00093E0A0E0B0E080936C0190936D01A0935B
:100ED0006E01B0936F0187E191E090936901809377
:100EE00068018FEF9FEF9093750180937401C8EBB9
:100EF000D1E00CEB11E0A12CB12C9924939489E260
:100F0000C82E81E0D82E91EC892ED8019C92F50153
:100F1000E854FE4F7F019582CE010B969F838E830E
:100F200019861886D982C8829486958683860E94FF
:100F30002402FC012181D8018C9190E0820F911D47
:100F40000897BCF0B2E1AB0EB11C62960E5E1F4F6B
:100F5000E4E2AE16B104C9F6DF91CF911F910F9173
:100F6000FF90EF90DF90CF90BF90AF909F908F90C9
:100F70000895A281B381109719F4D383C2830CC062
:100F800018968D919C911997009711F0DC01F8CF7C
:100F90001996DC93CE9318978081D80112978C9381
:100FA000818111968C939081D70115968C91890F30
:100FB000808380E0D8019C91891720F69181A92F28
:100FC000B0E0AD01445F5E4F2E813F81280F311D9F
:100FD000D9012C91DA012C939F5F91838F5FEACF27
:100FE000789484B5826084BD84B5816084BD85B504
:100FF000826085BD85B5816085BD80916E00816010
:1010000080936E00109281008091810082608093B5
:1010100081008091810081608093810080918000B7
:101020008160809380008091910082608093910024
:101030008091910081608093910080919000816007
:10104000809390008091C10084608093C100809162
:10105000C10082608093C1008091C1008160809353
:10106000C1008091C30081608093C3008091C00063
:1010700082608093C0008091C20081608093C20032
:1010800080917A00846080937A0080917A008260F7
:1010900080937A0080917A00816080937A008091B9
:1010A0007A00806880937A001092670110925C0148
:1010B00010925B018091D70081608093D70080EA15
:1010C0008093D80089B5806189BD89B5826089BD6A
:1010D00009B400FEFDCF61E070E080E090E00E9486
:1010E0008F028091D8008F7C80618093D80080919E
:1010F000E000807F8093E0008091E1008E7E80930D
:10110000E1008DE08093E200559A209AEEEFFFE730
:10111000859194918B3F9C4D19F481E080935A0105
:101120008AB1807F8AB98BB18F608BB980B38F70A1
:1011300080BB81B3806F81BB8AB18F768AB98BB156
:1011400080698BB985B18A6085B984B18A6084B9B8
:1011500064E670E080E090E00E948F0212E0CBE451
:10116000D0E00AE082E1F82E109262011092630151
:10117000109264011092650185B1812785B9CE0175
:101180000197F1F789B18F7090916201892B80935B
:1011900062013FB1632F62956F706093640185B106
:1011A000802785B9CE010197F1F789B18F708093BF
:1011B00063019FB1292F22952F702093650195B16E
:1011C000957F95B9FE013197F1F749B190E1499FBB
:1011D000A00111245527FA01E82BCF018093630168
:1011E0009FB1907F922B9093650125B12A6025B91C
:1011F000FE013197F1F729B1F0E12F9F9001112401
:10120000332740916201242B209362013FB1307F4C
:10121000362B209520936201809580936301832F64
:10122000809580936401909590936501109261017F
:10123000E090610121E02E1508F496CF8E2D90E00C
:101240009C01220F331FD901AE59BE4F4C91F901B9
:10125000E35AFE4F5081451305C011966C915181A0
:101260006517D9F1F901EE59FE4F5181F89EB00191
:10127000F99E700D1124FB01EA53FE4F842F8078F4
:1012800090E0880F991F852B8083818190FB80F9E6
:101290008183DB01A854BE4F41FB882780F9942F3E
:1012A0009170891B51968C93519743FB882780F945
:1012B00042FB992790F9891B50968C935097F9011E
:1012C000E35AFE4F408351836A537E4F13968C91AD
:1012D00044E050E080640E94C902E394E09261011E
:1012E000A7CFEE0FFF1F0590F491E02D099481E048
:1012F00090E0F8940C948309FB01DC0101900D92BD
:0A1300000020E1F70895F894FFCFF4
:10130A00FFFFFFFF00E100000000000000C1808134
:10131A00000000000000002B016303120241018E4D
:10132A00014C016A01000000007903BE03A0030D0D
:10133A000453415455524E20746F205553420000B5
:2070000055C000006EC000006CC000006AC0000068C0000066C0000064C0000062C0000043
:2070200060C000005EC00000F2C400005AC0000058C0000056C0000054C0000052C00000EE
:2070400050C0000078C000004CC000004AC0000048C0000046C0000044C0000042C00000BE
:2070600040C000003EC000003CC000003AC0000038C0000036C0000034C0000032C0000048
:2070800030C000002EC000002CC000002AC0000028C0000026C0000024C0000022C00000A8
:2070A00020C000001EC000001CC0000011241FBECFEFDAE0DEBFCDBF11E0A0E0B1E0E2E3BC
:2070C000FFE702C005900D92A83AB107D9F711E0A8EAB1E001C01D92AE3BB107E1F78FD30B
:2070E00026C78ECFF89410926F0010928100109285001092840081E085BF15BE47985D9AEB
:20710000289A0C94000008952091B2013091B3012F5F3F4F3093B3012093B201932F37FFA6
:2071200003C08EEF831B982F990F921710F447980895479A08951F920F920FB60F9211246E
:207140002F938F939F93EF93FF9310928500109284008091A8019091A901009741F00197D3
:207160009093A9018093A801892B09F45D9A8091AA019091AB01009741F001979093AB0126
:207180008093AA01892B09F4289AE0E0F0E0859194918F5F9F4F49F08091AC019091AD0151
:2071A00001969093AD018093AC01FF91EF919F918F912F910F900FBE0F901F90189584E0BC
:2071C0008093E9000DC08091E8008B778093E80003C08EB3882351F08091E80082FFF9CFBE
:2071E0008091E80085FFEFCF8091F1000895982F83E08093E9008091E80085FD0DC0809136
:20720000E8008E778093E80003C08EB3882369F08091E80080FFF9CF9093F1005D9884E6CB
:2072200090E09093A9018093A80108954F925F926F927F928F929F92AF92BF92CF92DF921E
:20724000EF92FF920F931F93CF93DF9384E08093E9008091E80082FF57C2289884E690E067
:207260009093AB018093AA01AADF182F853481F48CE49DE19093AD018093AC0107B600FC4B
:20728000FDCFF999FECF81E180935700E89503C0843519F494DF8DE00DC28C34E1F38035F9
:2072A000D1F3843721F484E4A2DF80E003C2813611F489E5FFC18134B1F481DF182F7FDFE3
:2072C00090E0880F991FAA2797FDA095BA2F312F330F20E0442737FD4095542F822B932B68
:2072E000A42BB52BB8C1803711F483E5E3C1833549F4C0E0D1E089917ADF21E0C730D20714
:20730000D1F7D9C1863521F481E371DF80E3D2C1833731F487E86BDF85E969DF8EE1CAC149
:207320008536B9F4E0E0F0E093E085E090935700E89507B600FCFDCF80935700E89507B65D
:2073400000FCFDCFE058FF4FA0E7E030FA0771F7A2CF823739F4E1E0F0E089E08093570024
:207360008491A8C1863439F4E0E0F0E089E08093570084919FC18E3439F4E3E0F0E089E0E5
:2073800080935700849196C1813539F4E2E0F0E089E08093570084918DC1823631F489E521
:2073A00026DF80E024DF80E885C1823419F0873609F0E5C01092AD011092AC0100DF082FE8
:2073C000FEDEF82EFCDE682E8554823008F071C1902F80E0CF2DD0E0C82BD92B10926F00B3
:2073E000173609F04BC081E180935700E895DD24CC24C3943FC0E090AE01F090AF010091CC
:20740000B0011091B101B6E46B16D9F4ED2DF0E0EE29FF29E4918E2FEADEDD2081F082E08D
:2074200090E0A0E0B0E0E80EF91E0A1F1B1FE092AE01F092AF010093B0011093B101DC2470
:2074400018C0D801C701B695A7959795879559D5CEDE82E090E0A0E0B0E0E80EF91E0A1FF2
:207460001B1FE092AE01F092AF010093B0011093B1012197209709F0BECF7DC08090AE01F5
:207480009090AF01A090B001B090B10196E4691609F05DC083E0F40180935700E89507B63E
:2074A00000FCFDCF54C0F6E46F1661F5772031F1E090AE01F090AF010091B0011091B1019E
:2074C0007EDED82ECC24852D90E08C299D29F7010C0140925700E895112482E090E0A0E08B
:2074E000B0E0E80EF91E0A1F1B1FE092AE01F092AF010093B0011093B10102C060DE582E1A
:20750000742423C0E090AE01F090AF010091B0011091B10116950795F794E79450DE682FFA
:20752000C701F7D48091AE019091AF01A091B001B091B1010296A11DB11D8093AE01909349
:20754000AF01A093B001B093B101219704C05524772444244394209709F0A5CF96E46916B6
:2075600041F485E0F40180935700E89507B600FCFDCF8DE03CDE82E080936F009CC0833492
:2075800071F40091AE011091AF0119DE90E021E0F8010C0120935700E89511247CCE8336C8
:2075A00019F5E090AE01F090AF010091B0011091B10105DEF701E16090E021E00C0120938C
:2075C0005700E895112482E090E0A0E0B0E0E80EF91E0A1F1B1FE092AE01F092AF0100936A
:2075E000B0011093B10157CE8D3661F4E091AE01F091AF0185E080935700E89507B600FCF2
:20760000FDCF49CE823551F4E091AE01F091AF0105911491812FEBDD802F4CC0843421F5FE
:20762000E090AE01F090AF010091B0011091B10116950795F794E794C2DD682FC70169D4DE
:207640008091AE019091AF01A091B001B091B1010296A11DB11D8093AE019093AF01A093D8
:20766000B001B093B10117CE843609F5E090AE01F090AF010091B0011091B101D801C70142
:20768000B695A795979587953CD4B1DD82E090E0A0E0B0E0E80EF91E0A1F1B1FE092AE010A
:2076A000F092AF010093B0011093B10104C08B3111F08FE39CDD83E08093E9009091E8002B
:2076C0008091E8008E778093E80095FF04C010C08EB38823C9F08091E80080FFF9CF809193
:2076E000E8008E778093E80003C08EB3882361F08091E80080FFF9CF84E08093E9008091F1
:20770000E8008B778093E800DF91CF911F910F91FF90EF90DF90CF90BF90AF909F908F90AC
:207720007F906F905F904F9008959091B601892F8F77813249F58091B7018032A1F081328A
:2077400019F5913A09F58091E800877F8093E8008DE091E067E070E00BD28091E8008B770B
:207760008093E8000895913279F48091E800877F8093E8008DE091E067E070E05DD2809192
:20778000E8008E778093E800089582E061EC42E0B5D083E061E842E1B1D084E060E842E1EF
:2077A000ADC084B7877F84BF88E10FB6F89480936000109260000FBE20E880E090E00FB63F
:2077C000F89420936100809361000FBE81E085BF92E095BF3F9A209A559AE1E6F0E02083A1
:2077E000108247985D9A289A109289008AEF8093880090936F0083E080938100F0C0409116
:20780000000850910108109201081092000894B714BE88E10FB6F8948093600010926000D5
:207820000FBE292F30E0F901E270F07091FD18C090FF05C0859194918F5F9F4F81F423FFFF
:207840000FC08091090190910A014817590741F0E0E0F0E0859194918F5F9F4F09F042DC64
:20786000A0DF78941092AD011092AC010CC0DEDC36D38091AC019091AD0181549F4110F00D
:207880001092140141DC80911401882381F78091E00081608093E00025DC80E090E0089598
:2078A000FA01923049F0933061F09130F9F485E191E022E130E01EC087E291E02EE330E04D
:2078C00019C0882329F485E691E024E030E012C0813029F489E691E022E230E00BC0823006
:2078E00029F48DE891E028E130E004C080E090E020E030E091838083C90108958093E9004E
:207900008091EB0081608093EB001092ED006093EC004093ED008091EE00881F8827881F62
:2079200008958091B60188238CF403C08EB38823B1F08091E80082FFF9CF8091E8008B772A
:207940008093E80008958EB3882349F08091E80080FFF9CF8091E8008E778093E800089594
:20796000EF92FF920F931F9345D04CD008ED10E0F80180818F77808380818068808380819B
:207980008F7D808319BC1EBA1092B40180EEE82EF12CF70180818B7F8083F8018081816052
:2079A000808380E060E042E0A9DFE1EEF0E080818E7F8083E2EEF0E0808181608083808144
:2079C00088608083F70180818E7F8083F8018081806180831F910F91FF90EF900895E7ED06
:2079E000F0E08081816080838AE482BF81E08093B501B6CFE8EDF0E080818E7F808310921C
:207A0000E20008951092DA001092E10008951F920F920FB60F9211242F933F934F935F93F6
:207A20006F937F938F939F93AF93BF93EF93FF938091DA0080FF1BC08091D80080FF17C0B2
:207A40008091DA008E7F8093DA008091D90080FF0BC080E189BD82E189BD09B400FEFDCF36
:207A600081E08EBB3BD203C019BC1EBA37D28091E10080FF17C08091E20080FF13C0809138
:207A8000E2008E7F8093E2008091E20080618093E2008091D80080628093D80019BC85E049
:207AA0008EBB1CD28091E10084FF2CC08091E20084FF28C080E189BD82E189BD09B400FEC5
:207AC000FDCF8091D8008F7D8093D8008091E1008F7E8093E1008091E2008F7E8093E20012
:207AE0008091E20081608093E2008091B401882331F48091E30087FD02C081E001C084E067
:207B00008EBBECD18091E10083FF21C08091E20083FF1DC08091E100877F8093E10082E06A
:207B20008EBB1092B4018091E1008E7F8093E1008091E2008E7F8093E2008091E2008061E9
:207B40008093E20080E060E042E0D8DEC7D1FF91EF91BF91AF919F918F917F916F915F9130
:207B60004F913F912F910F900FBE0F901F9018959C014091BC015091BD014617570718F49D
:207B8000F90190E044C06115710511F0AB01F8CF8091E8008E778093E80040E050E0F0CF0F
:207BA0008EB3882309F444C0853009F443C08091E80083FF02C081E008958091E80082FD70
:207BC00031C08091E80080FF22C08091F3009091F200782F60E0292F30E0262B372B07C07A
:207BE00081918093F100415050402F5F3F4F4115510519F02830310598F390E02830310566
:207C000009F491E08091E8008E778093E8004115510531F6992321F605C08EB3882341F075
:207C2000853041F08091E80082FFF7CF80E0089582E0089583E008959C016115710529F47C
:207C40008091E8008B778093E800F90126C08EB3882391F1853091F18091E80083FF02C06C
:207C600081E008958091E80082FFF1CF06C08091F10081936150704059F02091F300809191
:207C8000F200322F20E090E0822B932B892B79F78091E8008B778093E80061157105B9F601
:207CA00005C08EB3882341F0853041F08091E80080FFF7CF80E0089582E0089583E00895C2
:207CC0000F931F93DF93CF9300D0CDB7DEB7E6EBF1E08091F100819381E0EE3BF807C9F792
:207CE00024DD8091E80083FFE4C08091B6019091B701953009F46DC0963040F4913081F1A7
:207D0000913070F0933009F0D4C02AC0983009F4A3C0993009F4B2C0963009F0CAC07CC023
:207D2000803809F4C6C0823809F0C3C08091BA0187708093E9008091EB001092E9002091DB
:207D4000E800277F2093E80090E025E0969587952A95E1F781708093F1001092F10087C0D8
:207D6000882319F0823009F0A4C08F71823009F0A0C08091B801882331F52091BA01277097
:207D800009F497C02093E9008091EB0080FF1BC0933021F48091EB00806213C08091EB0018
:207DA00080618093EB0081E090E002C0880F991F2A95E2F78093EA001092EA008091EB00E5
:207DC00088608093EB001092E9008091E800877F51C0882309F06DC01091B8011F770FB79B
:207DE000F8948091E800877F8093E8009ADD8091E80080FFFCCF8091E3008078812B809398
:207E0000E30080688093E300112311F482E001C083E08EBB0FBF4DC08058823008F049C033
:207E20008091B8019091B9016091BA01AE014F5F5F4F36DDBC01009709F43BC08091E8008E
:207E4000877F8093E80089819A8192DE8091E8008B778093E8002DC0803859F58091E800AA
:207E6000877F8093E8008091B4018093F1008091E8008E778093E80054DD1BC08823C9F4CA
:207E80009091B8019230A8F48091E800877F8093E8009093B40145DD8091B401882331F420
:207EA0008091E30087FD02C081E001C084E08EBB6CDC8091E80083FF0AC08091EB0080624E
:207EC0008093EB008091E800877F8093E8000F900F90CF91DF911F910F91089508951F9360
:207EE0008EB3882361F01091E9001092E9008091E80083FF01C0E4DE17701093E9001F916F
:207F00000895F999FECF92BD81BDF89A992780B50895262FF999FECF1FBA92BD81BD20BDBD
:207F20000FB6F894FA9AF99A0FBE01960895F894FFCF4341544552494E4100777700080031
:207F40000000000000080112011001020000084123360001000201000109023E00020100FF
:207F600080320904000001020201000524001001042402040524060001070582030800FF0C
:207F800009040100020A000000070504021000010705830210000104030904220341007216
:207FA000006400750069006E006F0020004C0065006F006E006100720064006F0000001836
:1A7FC00003410072006400750069006E006F0020004C004C004300000000D7
:00000001FF
